:100000000FC03BC027C026C025C025C123C022C0C9
:1000100021C020C0ADC01EC01DC01CC01BC012012D
:1000200011241FBECFE5D2E0DEBFCDBF20E0A0E6A9
:10003000B0E001C01D92AA37B207E1F710E0C0E1BD
:10004000D0E003C02197FE0165D1CF30D107D1F7B1
:10005000EDD066C1D5CFF89482E08ABD85E889BD30
:1000600081E083BF90E199BF97BB9BE098BB20E6FE
:100070002BBF95BB85BF789408951F920F920FB642
:100080000F9211240F931F932F933F934F935F93DE
:100090006F937F938F939F93AF93BF93EF93E09171
:1000A00060004091690050916A0060916B0070910E
:1000B0006C008091610090916200A0916300B0910A
:1000C00064000091650010916600209167003091F6
:1000D0006800E3FD16C0840F951FA61FB71F801B85
:1000E000910BA20BB30BB695A79597958795809327
:1000F000610090936200A0936300B0936400019745
:1001000019C0E0916000840F951FA61FB71F801BC8
:10011000910BA20BB30B22E0B695A7959795879507
:100120002A95D1F78093610090936200A0936300B9
:10013000B09364009093700080936F0040936500CB
:10014000509366006093670070936800EF91BF91D1
:10015000AF919F918F917F916F915F914F913F915F
:100160002F911F910F910F900FBE0F901F90189518
:100170001F920F920FB60F9211242F933F938F93DC
:100180009F93AF93BF938091690090916A00A09173
:100190006B00B0916C000196A11DB11D80936900A8
:1001A00090936A00A0936B00B0936C0020916D0057
:1001B00030916E0080916F0090917000B0990BC0EB
:1001C0008217930744F410926E0010926D0098B35A
:1001D00080E1892788BB80916D0090916E00019627
:1001E00090936E0080936D0080916000909160000C
:1001F00021E093FB992790F9921304C086958170B2
:10020000821711F081E001C083E085BFBF91AF91FB
:100210009F918F913F912F910F900FBE0F901F9044
:100220001895089586B380936000089581B781BFC3
:100230005CD011DFF6DFFECF80B7807F80BF80B754
:10024000806880BF8CB580648CBD8FEF8DBD80B71A
:10025000876080BF08951F920F920FB60F921124EE
:100260002F933F938F939F93AF93BF93809172008F
:1002700090917300A0917400B0917500309171005D
:1002800026E0230F2D3730F029E8230F0396A11D18
:10029000B11D03C00296A11DB11D20937100809372
:1002A000720090937300A0937400B09375008091D6
:1002B000760090917700A0917800B0917900019636
:1002C000A11DB11D8093760090937700A0937800D4
:1002D000B0937900BF91AF919F918F913F912F91F2
:1002E0000F900FBE0F901F9018958AB582608ABD3F
:1002F0008AB581608ABD83B7887F836083BF789425
:1003000089B7826089BF98DF86B18877866886B9A9
:10031000379A0895EE0FFF1F0590F491E02D099490
:04032000F894FFCF7F
:00000001FF
